:020000040800F2
:100000000050002021020008552800085928000847
:100010005D2800086128000865280008000000002D
:100020000000000000000000000000006928000837
:100030006D280008000000007128000875280008DD
:100040007923000879230008792300087923000820
:100050007923000879230008792300087923000810
:100060007923000879230008792300087923000800
:1000700079230008792300087923000879230008F0
:1000800079230008792300087923000879230008E0
:1000900079230008792300087923000879230008D0
:1000A00079230008792300087923000879230008C0
:1000B00079230008792300087923000879230008B0
:1000C00079230008792300087923000879230008A0
:1000D0007923000879230008792300087923000890
:1000E0007923000879230008792300080000000024
:1000F0000000000000000000000000000000000000
:1001000000000000000000005FF808F100B583B0B7
:1001100002F09AF8304B314A1360314A1360314B88
:10012000314A03E011681960043304322F498B42CD
:10013000F8D32A4B1A682E4B9A4204D1284B1A68DE
:100140002C4B9A4200D0FEE7234B2B4A13602B4ADC
:1001500013602B4B02E000221A600433294A9342B9
:10016000F9D3254B1B6813B9244B1B6803B1FEE779
:1001700002F076F8694601A802F010F8224C234BF1
:100180001C1BA410002504E01F4B53F82530984792
:100190000135AC42F8DC1E4C1E4B1C1BA410002584
:1001A00004E01B4B53F8253098470135AC42F8DC8E
:1001B0000099019802F070FA0546174C174B1C1B6A
:1001C000A41004E0013C144B53F824309847002C51
:1001D000F8DC284601F0BEFFBABADECA00000020F3
:1001E0008000002000000020EC3A0008840000207D
:1001F0007856341232547698840000201803002078
:10020000840000201C030020780300087803000805
:1002100078030008780300087803000878030008D2
:1002200008B5FFF773FF00BF00BEFEE71EF0040F26
:100230000CBFEFF30880EFF309807146414A104785
:100240002DE9F04182B004468846134B5E6B9F6BEC
:100250009D6A1B6B13F0020F0DD00F4BDB6A002B56
:1002600009DA4BF6AB6102F077F820B14FF00042AB
:10027000094BDA620CE0094801F098FFCDF80080E4
:100280003B4632462946204601F0EEFF00BEFEE71F
:1002900002B0BDE8F08100BF00ED00E05C3A00086C
:1002A00000BEFEE71EF0040F0CBFEFF30880EFF373
:1002B00009807146244A10472DE9F04182B0044676
:1002C0008846084B5E6B9F6B9D6A074801F06EFF86
:1002D000CDF800803B4632462946204601F0C4FF57
:1002E00000BEFEE700ED00E06C3A00081EF0040FCF
:1002F0000CBFEFF30880EFF309807146134A1047F3
:100300002DE9F04182B004468846084B5E6B9F6B36
:100310009D6A074801F04AFFCDF800803B4632460F
:100320002946204601F0A0FF00BEFEE700ED00E0F8
:10033000783A000800BEFEE700BEFEE700BEFEE71A
:100340007047000041020008B902000801030008DC
:10035000EC3A00080000002084000020EC3A00087D
:100360000000000000000000840000201C030020AA
:08037000000000000000000085
:1003780010B5044601F0ACF8064BA3FB0030800929
:1003880000F09CF9002221464FF0FF3000F054F9AC
:10039800002010BDD34D621008B5074A136843F01A
:1003A80010031360032000F029F90020FFF7E0FF95
:1003B80002F084F9002008BD00200240024A1368B8
:1003C80001331360704700BF88000020014B186894
:1003D800704700BF8800002010B582B00190FFF779
:1003E800F5FF0446FFF7F2FF001B019B9842F9D383
:1003F80002B010BD002800F0FB8038B50446026842
:100408007C4B9A4203D0B8217B4802F055F9A36986
:10041800012B03D9B921784802F04EF9E369012B81
:1004280003D9BA21744802F047F9236A012B03D98A
:10043800BB21714802F040F9636A012B03D9BC2142
:100448006D4802F039F9A36A012B03D9BD216A4826
:1004580002F032F9E36A012B03D9BE21664802F0A3
:100468002BF9A36863B1B3F1804F09D0B3F1004F02
:1004780006D0B3F1404F03D0BF215F4802F01CF90A
:10048800E36863B1B3F1807F09D0B3F1007F06D090
:10049800B3F1407F03D0C021574802F00DF923691A
:1004A800B3F5702F03D9C121534802F005F96369E8
:1004B800B3F5E00F03D9C2214F4802F0FDF8636895
:1004C800013BB3F5806F03D3C3214B4802F0F4F826
:1004D80094F8393013F0FF0F05D1002384F8383031
:1004E800204602F033F9022384F839302268136871
:1004F80023F0020313602268136843F001031360BA
:10050800FFF764FF05460BE0FFF760FF401B0A2872
:1005180006D9032084F83900002384F8383038BD20
:1005280023685A6812F0010FEED05A6812F0010FD2
:100538004FD0A269012A01D0002100E08021E269A0
:10054800012A01D141F04001226A012A01D141F07A
:100558002001626A012A01D141F01001A26A012A30
:1005680001D141F00801E26A012A01D141F00401F8
:100578001A6822F0FC020A431A602168A268E3683C
:100588001A4323691A4363691A436368013B134397
:10059800CB612268136823F001031360FFF716FF8D
:1005A80005460BE0FFF712FF401B0A2806D9032077
:1005B80084F83900002384F8383038BD23685A6835
:1005C80012F0010FEED05B6813F0010F03D1002386
:1005D80002E0002300E001232BB10020E0630123A7
:1005E80084F8393038BD042384F83930012038BD07
:1005F80001207047006400401838000810B5044610
:10060800C31E042B03D9BA21094802F055F8094A38
:10061800D36823F4E0631B041B0C240204F4E06495
:10062800234343F0BF6343F40033D36010BD00BFDE
:100638004438000800ED00E070B504460E46154643
:100648000F2A03D9D2211A4802F036F80F2E03D9FF
:10065800D321174802F030F8164BDA68C2F30222A9
:10066800C2F10701042928BF0421131D062B01D953
:10067800033A00E00022012303FA01F10139314075
:10068800914003FA02F2013A2A400A43002C06DAA2
:1006980004F00F041201D2B2074B1A5570BD1201B3
:1006A800D2B204F1604404F5614484F8002370BDBB
:1006B8004438000800ED00E014ED00E00138B0F126
:1006C800807F0AD2064B5860F021064A82F8231030
:1006D8000020986007221A6070470120704700BF09
:1006E80010E000E000ED00E010B50446042805D055
:1006F80020B14FF4DF71084801F0DEFF042C05D16A
:10070800064A136843F00403136010BD034A1368D4
:1007180023F00403136010BD4438000810E000E023
:1007280008B502F059F908BD2DE9F04383B08046B9
:100738000F46AE4B984213D003F5806398420FD012
:1007480003F5806398420BD003F58063984207D085
:1007580003F58063984203D0CF21A54801F0ACFF90
:100768003B881BB9D021A24801F0A6FF7B68012B6A
:1007780022D9112B20D0022B1ED0122B1CD09D4A1F
:10078800934219D002F58012934215D002F58012D7
:10079800934211D0A2F5F81293420DD002F58012BF
:1007A800934209D002F58012934205D0032B03D05F
:1007B800D1218F4801F080FF4FF000094E462BE110
:1007C8000125B5403C682C40A54240F02481874B68
:1007D800984513D003F5806398450FD003F58063DF
:1007E80098450BD003F58063984507D003F58063DF
:1007F800984503D0DF217E4801F05EFF7B68122B0D
:1008080049D00CD8022B3AD004D8002B4FD0012B5A
:100818001ED067E0032B60D0112B24D062E0764A0B
:10082800934244D008D8A2F5801293423FD002F5F3
:100838008032934256D13AE0704A934237D002F55B
:100848008032934233D0A2F5801293424AD12EE0EF
:10085800FB68013B022B03D9E721654801F02CFF17
:10086800D7F80C903EE0FB68013B022B03D9EE2140
:100878005F4801F021FFFB6803F1040932E0FB68DF
:10088800013B022B03D9F521594801F015FFFB68FC
:1008980003F1080926E0FB68013B022B03D9FC2180
:1008A800534801F009FFFB6803F10C091AE0BB6823
:1008B800022B04D940F209114D4801F0FDFEBB6836
:1008C80073B1012B04D1C8F810504FF0080909E0A2
:1008D800C8F814504FF0080904E04FF0000901E08F
:1008E8004FF00409FF2C01D8404601E008F104004C
:1008F800FF2C01D8B30002E0A6F108039B000168B1
:100908000F229A4021EA020209FA03F31343036013
:100918007B6813F0805F7ED0394B9A6942F0010200
:100928009A619B6903F001030193019BB1088A1C3A
:10093800344B53F8222006F003039B000F20984005
:1009480022EA0000294A90450DD002F580629045C0
:100958000BD002F58062904509D002F5806290457F
:1009680007D1032206E0002204E0012202E002226D
:1009780000E0042202FA03F303430231214A42F859
:1009880021307B6813F4803F05D002F5806213683C
:100998002343136004E01C4A136823EA040313602A
:1009A8007B6813F4003F04D0174A5368234353600D
:1009B80004E0154A536823EA040353607B6813F480
:1009C800801F04D0104A93682343936004E00E4AC2
:1009D800936823EA040393607B6813F4001F15D01F
:1009E800094AD3681C43D46015E000BF00080140E1
:1009F80074380008000011100000211000003110A8
:100A0800001002400000014000040140054AD3687C
:100A180023EA0404D46001360F2E7FF6D1AE03B06A
:100A2800BDE8F0830004014070B5064615460C4643
:100A380021B94FF4F271084801F03EFE012D04D9A6
:100A480040F2E511044801F037FE0DB1346170BD84
:100A58002404346170BD00BF7438000838B50446FA
:100A68000D4621B94FF4FD71034801F025FEE168F8
:100A78006940E16038BD00BF7438000830B583B004
:100A8800044620B94FF48771B94801F015FE236870
:100A98003BB113F00F0F04D140F20F11B44801F02D
:100AA8000BFE236813F0010F00F0A380636853B1B5
:100AB800B3F5803F07D0B3F5A02F04D040F215114D
:100AC800AB4801F0F9FDAB4B5B6803F00C03042B5A
:100AD8000AD0A84B5B6803F00C03082B1BD1A54B6D
:100AE8005B6813F4803F16D04FF4003393FAA3F3F6
:100AF800A04B1A684FF4003393FAA3F3B3FA83F3C5
:100B080003F01F0322FA03F313F0010F71D0636897
:100B1800002B6ED11BE36368B3F5803F05D1954A7E
:100B2800136843F48033136026E063B903F180430C
:100B380003F504331A6822F480321A601A6822F422
:100B480080221A6018E0B3F5A02F0CD103F180437E
:100B5800A3F53C331A6842F480221A601A6842F4FA
:100B680080321A6008E0834B1A6822F480321A60D7
:100B78001A6822F480221A606368EBB1FFF726FC3A
:100B8800054605E0FFF722FC401B642800F2E182DD
:100B98004FF4003393FAA3F3764B1A684FF40033FB
:100BA80093FAA3F3B3FA83F303F01F0322FA03F3D0
:100BB80013F0010FE6D01CE0FFF708FC054605E03E
:100BC800FFF704FC401B642800F2C5824FF4003391
:100BD80093FAA3F3674B1A684FF4003393FAA3F31D
:100BE800B3FA83F303F01F0322FA03F313F0010FA0
:100BF800E6D1236813F0020F00F0A0802369012BCF
:100C080004D940F249115A4801F056FD63691F2B77
:100C180004D94FF4A571564801F04EFD554B5B6859
:100C280013F00C0F0AD0534B5B6803F00C03082B2E
:100C380027D1504B5B6813F4803F22D1022393FAEB
:100C4800A3F34C4B1A68022393FAA3F3B3FA83F382
:100C580003F01F0322FA03F313F0010F03D02369F3
:100C6800012B40F07A824348036823F0F801636956
:100C7800F82292FAA2F2B2FA82F293400B4303608E
:100C88005CE023699BB3012292FAA2F3B3FA83F3DF
:100C98009B0003F1844303F584031A60FFF796FB76
:100CA800054605E0FFF792FB401B022800F2578239
:100CB800022393FAA3F32F4B1A68022393FAA3F3A0
:100CC800B3FA83F303F01F0322FA03F313F0010FBF
:100CD800E8D02848036823F0F8016369F82292FAFB
:100CE800A2F2B2FA82F293400B43036026E001239A
:100CF80093FAA3F3B3FA83F39B0003F1844303F558
:100D0800840300221A60FFF761FB054605E0FFF740
:100D18005DFB401B022800F22482022393FAA3F30E
:100D2800144B1A68022393FAA3F3B3FA83F303F07C
:100D38001F0322FA03F313F0010FE8D1236813F01D
:100D4800080F5CD0A369012B04D94FF4C57108487A
:100D580001F0B2FCA3696BB3012292FAA2F3B3FAD1
:100D680083F3054941F82320FFF730FB05460BE0E4
:100D7800B83800080010024080044242FFF726FB02
:100D8800401B022800F2EF81022393FAA3F293FAA0
:100D9800A3F2A44A526A93FAA3F3B3FA83F303F0D3
:100DA8001F0322FA03F313F0010FE7D00120FFF726
:100DB80013FB24E0012393FAA3F3B3FA83F300218E
:100DC800994A42F82310FFF701FB054605E0FFF7B3
:100DD800FDFA401B022800F2C881022393FAA3F20D
:100DE80093FAA3F28F4A526A93FAA3F3B3FA83F3FE
:100DF80003F01F0322FA03F313F0010FE7D123686E
:100E080013F0040F00F0AB80E368012B06D9052B23
:100E180004D040F2B711854801F04EFC814BDA69E5
:100E280042F08052DA61DB6903F080530193019B41
:100E38007F4A136843F480731360FFF7C7FA0546C7
:100E480005E0FFF7C3FA401B642800F29081784B55
:100E58001B6813F4807FF4D0E368012B05D1714A35
:100E6800136A43F00103136222E063B903F180437C
:100E780003F504331A6A22F001021A621A6A22F090
:100E880004021A6214E0052B09D1664B1A6A42F073
:100E980004021A621A6A42F001021A6208E0614BFF
:100EA8001A6A22F001021A621A6A22F004021A620D
:100EB800E36853B3FFF78AFA054607E0FFF786FAB7
:100EC800401B41F28833984200F25381022393FA7F
:100ED800A3F293FAA3F3B3FA83F35B0943F0020393
:100EE800DBB2022B02D14F4B1A6A01E04D4B5A6A12
:100EF800022393FAA3F3B3FA83F303F01F0322FA4E
:100F080003F313F0010FD9D029E0FFF75FFA054684
:100F180007E0FFF75BFA401B41F28833984200F282
:100F28002A81022393FAA3F293FAA3F3B3FA83F381
:100F38005B0943F00203DBB2022B02D1394B1A6A78
:100F480001E0384B5A6A022393FAA3F3B3FA83F306
:100F580003F01F0322FA03F313F0010FD9D1E36959
:100F6800022B04D940F24721304801F0A5FBE36980
:100F7800002B00F002812B4A526802F00C02082A6A
:100F880000F0FD80022B40F0B780236A3BB1B3F537
:100F9800803F04D04FF41471244801F08DFB636A3C
:100FA80073B3B3F5802F2BD0B3F5002F28D0B3F54A
:100FB800402F25D0B3F5801F22D0B3F5A01F1FD036
:100FC800B3F5C01F1CD0B3F5E01F19D0B3F5001F4F
:100FD80016D0B3F5101F13D0B3F5201F10D0B3F5FA
:100FE800301F0DD0B3F5401F0AD0B3F5501F07D0FE
:100FF800B3F5601F04D040F251210C4801F05CFBAE
:101008004FF0807393FAA3F3B3FA83F39B0003F1D1
:10101800844303F5840300221A60FFF7D7F90546D5
:101028000EE000BF0010024080044242B8380008B9
:1010380000700040FFF7CAF9401B022800F2A180A7
:101048004FF0007393FAA3F3514B1A684FF00073F3
:1010580093FAA3F3B3FA83F303F01F0322FA03F31B
:1010680013F0010FE6D1236AB3F5803F10D1A368CE
:101078003BB1B3F5003F04D040F26721454801F089
:101088001BFB43494B6823F40032A36813434B60AE
:101098003F48436823F47411236A626A13430B437D
:1010A80043604FF0807393FAA3F3B3FA83F39B0082
:1010B80003F1844303F5840301221A60FFF786F9DC
:1010C800044604E0FFF782F9001B02285BD84FF0C2
:1010D800007393FAA3F32E4B1A684FF0007393FA38
:1010E800A3F3B3FA83F303F01F0322FA03F313F015
:1010F800010FE7D0002049E04FF0807393FAA3F383
:10110800B3FA83F39B0003F1844303F584030022BD
:101118001A60FFF75BF9044604E0FFF757F9001B74
:10112800022832D84FF0007393FAA3F3184B1A68C9
:101138004FF0007393FAA3F3B3FA83F303F01F039A
:1011480022FA03F313F0010FE7D100201EE001207B
:101158001CE003201AE0032018E0012016E0032019
:1011680014E0032012E0032010E003200EE0032027
:101178000CE003200AE0032008E0002006E001203C
:1011880004E0032002E0032000E0032003B030BDA8
:1011980000100240B838000830B486B01F4D02ACC9
:1011A80028686968AA68EB680FC42B8AADF8043010
:1011B8001B4B5B6803F00C02082A2AD103F4701158
:1011C8004FF4701292FAA2F2B2FA82F221FA02F203
:1011D80006A90A4412F8102C13F4803F15D0104BBE
:1011E8005B6803F400314FF4003393FAA3F3B3FAC6
:1011F80083F321FA03F306A90B4413F8140C094BE3
:10120800B3FBF0F000FB02F004E0074800FB02F03B
:1012180000E0044806B030BC704700BFA43800089E
:101228000010024000127A0000093D0070B50D461A
:10123800044620B94FF42F71A04801F03DFA236805
:1012480013F00F0F04D140F2BD219C4801F034FA8D
:10125800022D04D940F2BE21984801F02DFA984B8E
:101268001B6803F007039D420BD9954A136823F0C6
:1012780007032B431360136803F007039D4240F0F4
:101288000D81236813F0020F1DD0A368A3B1802B32
:1012980012D0902B10D0A02B0ED0B02B0CD0C02B7E
:1012A8000AD0D02B08D0E02B06D0F02B04D040F287
:1012B800D721824801F000FA82494B6823F0F002F6
:1012C800A36813434B60236813F0010F00F081807B
:1012D8006368022B04D940F2DE21784801F0ECF96A
:1012E8006268012A13D14FF4003393FAA3F3754BC4
:1012F80019684FF4003393FAA3F3B3FA83F303F0B6
:101308001F0321FA03F313F0010F28D1C8E0022AC2
:1013180013D14FF0007393FAA3F36A4B19684FF097
:10132800007393FAA3F3B3FA83F303F01F0321FACC
:1013380003F313F0010F12D1B4E0022393FAA3F3DD
:10134800604B1968022393FAA3F3B3FA83F303F00B
:101358001F0321FA03F313F0010F00F0A580594988
:101368004B6823F0030313434B60FFF72FF806463F
:101378006368012B0FD107E0FFF728F8801B41F2C3
:101388008833984200F292804E4B5B6803F00C035E
:10139800042BF1D11DE0022B16D107E0FFF716F858
:1013A800801B41F28833984200F28280454B5B688B
:1013B80003F00C03082BF1D10BE0FFF707F8801BB3
:1013C80041F28833984275D83E4B5B6813F00C0F96
:1013D800F3D13B4B1B6803F007039D420AD2384AFE
:1013E800136823F007032B431360136803F0070304
:1013F8009D4261D1236813F0040F19D0E36883B1CB
:10140800B3F5806F0DD0B3F5A06F0AD0B3F5C06FF8
:1014180007D0B3F5E06F04D040F23231274801F02D
:101428004BF928494B6823F4E062E36813434B60A7
:10143800236813F0080F1AD0236983B1B3F5806FBE
:101448000DD0B3F5A06F0AD0B3F5C06F07D0B3F5D0
:10145800E06F04D040F23931184801F02DF9194AEB
:10146800536823F46053216943EAC1035360FFF7CB
:1014780093FE144B5B6803F0F002F02393FAA3F396
:10148800B3FA83F322FA03F30F4AD35CD8400F4B25
:1014980018600020FEF76CFF002070BD012070BDB1
:1014A800012070BD012070BD012070BD032070BDFA
:1014B800032070BD032070BD012070BDB83800083E
:1014C8000020024000100240883A00080C0000206A
:1014D800014B1868704700BF0C00002010B4036A65
:1014E800046A24F001040462846924F0F00444EAE4
:1014F800021223F00A0319438261016210BC70478B
:1015080010B4036A23F0100303628469036A24F4A5
:10151800704444EA023223F0A00343EA01118261D5
:10152800016210BC704700BF836823F0700341F06C
:10153800070119438160704710B4846824F47F441C
:1015480042EA0323194344EA0103836010BC70474D
:101558002DE9F04104460D46036A23F001030362B6
:10156800066AD0F80480876927F073030F681F4361
:1015780026F002038E681E431C4B98420ED1CB689E
:1015880033B1082B04D041F21521194801F094F821
:1015980026F00806EB681E4326F00406134B9C420F
:1015A8001BD1AB69B3F5007F05D023B141F22221ED
:1015B8000F4801F081F86B69B3F5807F05D023B13E
:1015C80041F223210A4801F077F828F440786B6942
:1015D80048EA0308AB6948EA0308C4F80480A7612D
:1015E8006B6863632662BDE8F08100BF002C014090
:1015F800E43800082DE9F04104460E46036A23F456
:1016080080730362056AD0F80480C76927F0730302
:101618000F681F4325F400738D6843EA05251D4BA9
:1016280098420FD1CB6833B1082B04D041F2AA21DC
:10163800194801F041F825F40065F36845EA0325E7
:1016480025F48065134B9C421BD1B369B3F5007F29
:1016580005D023B141F2B7210F4801F02DF8736985
:10166800B3F5807F05D023B141F2B8210A4801F0D3
:1016780023F828F44058736948EA0318B36948EA1C
:101688000318C4F80480E7617368E3632562BDE862
:10169800F08100BF002C0140E43800082DE9F0413A
:1016A80004460F46036A23F480530362056AD0F8A0
:1016B8000480C66926F4E6430E6843EA062625F444
:1016C80000538D6843EA05350C4B98420ED14B699F
:1016D800B3F5807F05D023B141F2F521084800F029
:1016E800EBFF28F480487B6948EA8318C4F8048033
:1016F800E6617B6823642562BDE8F081002C014027
:10170800E438000810B504460368104A93420FD025
:10171800B3F1804F0CD0A2F59432934208D002F571
:101728008062934204D04FF49871094800F0C4FFD6
:10173800022384F839302268136843F001031360E8
:10174800012384F83930002010BD00BF002C01406F
:10175800E4380008704700BF38B590F83830012BDE
:1017680000F005820D460446012380F83830022334
:1017780080F839300B68B3F5805F16D0B3F5005F99
:1017880013D093B1102B10D0202B0ED0302B0CD0AF
:10179800402B0AD0502B08D0602B06D0702B04D0D9
:1017A80040F64B71A04800F087FF2268936823F445
:1017B8007F4323F0770393602B68402B00F0388138
:1017C8000ED8102B00F0828103D8002B00F0658121
:1017D800C6E1202B00F09381302B00F0A981BFE1F6
:1017E800702B28D006D8502B00F0B380602B00F067
:1017F800E580B5E1B3F5805F03D0B3F5005F61D054
:10180800AEE12368894A93420FD0B3F1804F0CD0E0
:10181800A2F59432934208D002F58062934204D034
:1018280040F65771804800F047FF2268936823F01C
:101838000703936094E123687C4A93420FD0B3F185
:10184800804F0CD0A2F59432934208D002F5806202
:10185800934204D04FF47661734800F02DFFAB68D3
:101868006BB1B3F5805F0AD0B3F5005F07D0B3F56D
:10187800405F04D040F663716B4800F01DFF6B6851
:10188800B3F5004F0AD04BB143B1022B06D00A2B57
:1018980004D040F66471644800F00EFFEB680F2B2B
:1018A80004D940F66571604800F006FFEB686A6885
:1018B800A9682068FFF740FE2268936843F0770321
:1018C80093604DE12368594A93420FD0B3F1804F9A
:1018D8000CD0A2F59432934208D002F5806293426C
:1018E80004D040F67A71504800F0E6FEAB686BB160
:1018F800B3F5805F0AD0B3F5005F07D0B3F5405F5A
:1019080004D040F67D71484800F0D6FE6B68B3F508
:10191800004F0AD04BB143B1022B06D00A2B04D09A
:1019280040F67E71404800F0C7FEEB680F2B04D9E3
:1019380040F67F713C4800F0BFFEEB686A68A96812
:101948002068FFF7F9FD2268936843F480439360A9
:1019580006E12368354A93420FD0B3F1804F0CD08B
:10196800A2F59432934208D002F58062934204D0E3
:1019780040F68E712C4800F09FFE6B68B3F5004F5F
:101988000AD04BB143B1022B06D00A2B04D040F643
:101998009171254800F090FEEB680F2B04D940F6B2
:1019A8009271214800F088FEEA6869682068FFF7AC
:1019B80095FD50212068FFF7B7FDD1E023681B4A49
:1019C80093420FD0B3F1804F0CD0A2F594329342DA
:1019D80008D002F58062934204D040F69D71124807
:1019E80000F06AFE6B68B3F5004F0AD04BB143B103
:1019F800022B06D00A2B04D04FF47A610A4800F073
:101A08005BFEEB680F2B04D940F6A171064800F085
:101A180053FEEA6869682068FFF772FD6021206854
:101A2800FFF782FD9CE000BFE4380008002C01406D
:101A38002368504A93420FD0B3F1804F0CD0A2F5DF
:101A48009432934208D002F58062934204D040F663
:101A5800AC71494800F030FE6B68B3F5004F0AD00E
:101A68004BB143B1022B06D00A2B04D040F6AF711C
:101A7800414800F021FEEB680F2B04D94FF47B613D
:101A88003D4800F019FEEA6869682068FFF726FDFE
:101A980040212068FFF748FD62E02368354A9342F9
:101AA8000FD0B3F1804F0CD0A2F59432934208D0F6
:101AB80002F58062934204D040F6BB712E4800F0D4
:101AC800FBFD00212068FFF72FFD49E02368294A24
:101AD80093420FD0B3F1804F0CD0A2F594329342C9
:101AE80008D002F58062934204D040F6C3712248C0
:101AF80000F0E2FD10212068FFF716FD30E02368B2
:101B08001C4A93420FD0B3F1804F0CD0A2F5943207
:101B1800934208D002F58062934204D040F6CB711C
:101B2800154800F0C9FD20212068FFF7FDFC17E0EB
:101B38002368104A93420FD0B3F1804F0CD0A2F51E
:101B48009432934208D002F58062934204D040F662
:101B5800D371094800F0B0FD30212068FFF7E4FC9C
:101B6800012384F83930002084F8380038BD022079
:101B780038BD00BF002C0140E43800080368184A4B
:101B880090420AD0B0F1804F07D0A2F5943290422B
:101B980003D002F58062904203D123F070034A68B3
:101BA80013430F4A90420AD0B0F1804F07D0A2F5F4
:101BB8009432904203D002F58062904203D123F41C
:101BC8004073CA68134303608B68C3620B688362FF
:101BD800034B984201D10B690363012343617047AA
:101BE800002C0140002845D010B504460368224A5D
:101BF80093420ED0B3F1804F0BD0A2F594329342AA
:101C080007D002F58062934203D0D7211B4800F029
:101C180053FDA3685BB1102B09D0202B07D0402BB4
:101C280005D0602B03D0D821144800F045FD236966
:101C38004BB1B3F5807F06D0B3F5007F03D0D9212F
:101C48000E4800F039FD94F8393013F0FF0F05D134
:101C5800002384F83830204600F0A6FD022384F8DB
:101C68003930211D2068FFF789FF012384F83930B6
:101C7800002010BD01207047002C0140E438000806
:101C8800002848D010B504460368244A93420FD070
:101C9800B3F1804F0CD0A2F59432934208D002F5EC
:101CA8008062934204D040F2E2311D4800F004FD06
:101CB800A36863B1102B0AD0202B08D0402B06D084
:101CC800602B04D040F2E331154800F0F5FC23699D
:101CD80053B1B3F5807F07D0B3F5007F04D04FF43C
:101CE80079710F4800F0E8FC94F8393013F0FF0FD1
:101CF80005D1002384F838302046FFF72BFD022356
:101D080084F83930211D2068FFF738FF012384F853
:101D18003930002010BD0120704700BF002C014061
:101D2800E43800082DE9F04104460F46036A23F021
:101D380010030362056AD0F80480866926F4E64336
:101D48000E6843EA062625F020038D6843EA051548
:101D58001C4B98420FD1CB6833B1082B04D041F209
:101D68005F21194800F0A8FC25F08005FB6845EACA
:101D7800031525F04005134B9C421BD1BB69B3F5F5
:101D8800007F05D023B141F26D210F4800F094FC8B
:101D98007B69B3F5807F05D023B141F26E210A48F3
:101DA80000F08AFC28F440687B6948EA8308BB692C
:101DB80048EA8308C4F80480A6617B68A3632562A7
:101DC800BDE8F081002C0140E438000890F8383074
:101DD800012B00F0E88070B516460D460446012335
:101DE80080F8383062B1042A0AD0082A08D00C2AB0
:101DF80006D0182A04D040F60D416C4800F05CFC6F
:101E08002B68602B06D0702B04D040F60E41674833
:101E180000F052FCAB6833B1022B04D040F60F41FE
:101E2800624800F049FC2B6933B1042B04D04FF40D
:101E380041615E4800F040FC022384F839300C2EE2
:101E480000F2AA80DFE806F007A8A8A82FA8A8A88B
:101E580058A8A8A880002368554A93420FD0B3F128
:101E6800804F0CD0A2F59432934208D002F58062DC
:101E7800934204D040F618414C4800F01DFC294616
:101E88002068FFF765FB2268936943F008039361B4
:101E98002268936923F004039361226891692B698E
:101EA8000B43936178E02368414A93420FD0B3F122
:101EB800804F0CD0A2F59432934208D002F580628C
:101EC800934204D040F62741384800F0F5FB2946F4
:101ED8002068FFF727FF2268936943F40063936142
:101EE8002268936923F4806393612268936929695E
:101EF80043EA012393614FE023682D4A93420FD0B0
:101F0800B3F1804F0CD0A2F59432934208D002F579
:101F18008062934204D040F63641244800F0CCFB5E
:101F280029462068FFF766FB2268D36943F0080357
:101F3800D3612268D36923F00403D3612268D1698D
:101F48002B690B43D36127E02368194A93420FD0CA
:101F5800B3F1804F0CD0A2F59432934208D002F529
:101F68008062934204D040F64541104800F0A4FB3B
:101F780029462068FFF792FB2268D36943F400637F
:101F8800D3612268D36923F48063D3612268D3695B
:101F9800296943EA0123D361012384F839300020F9
:101FA80084F8380070BD0220704700BFE43800088C
:101FB800002C014070B504460E461546164B984253
:101FC8000FD0B0F1804F0CD0A3F59433984208D0CD
:101FD80003F58063984204D041F2EB410F4800F0CA
:101FE8006BFB66B1042E0AD0082E08D00C2E06D042
:101FF800182E04D041F2EC41084800F05DFB0123A3
:1020080003FA06F2236A23EA02032362236AB5402D
:102018001D43256270BD00BF002C0140E438000854
:1020280038B504460D460368164A93420AD0B3F100
:10203800804F07D0A2F59432934203D002F5806214
:10204800934206D155B1042D08D0082D06D00C2D89
:1020580004D04FF488610C4800F02EFB0122294679
:102068002068FFF7A7FF2368064A934203D15A6CFA
:1020780042F400425A642268136843F00103136073
:10208800002038BD002C0140E438000838B504466B
:102098000D4603682B4A93420FD0B3F1804F0CD002
:1020A800A2F59432934208D002F58062934204D09C
:1020B80040F28C61244800F0FFFA2B6893B1102B92
:1020C80010D0202B0ED0302B0CD0402B0AD0502B08
:1020D80008D0602B06D0702B04D040F28D611A48CE
:1020E80000F0EAFA6B68802B05D023B140F28E61CC
:1020F800154800F0E1FA94F83830012B1FD001227E
:1021080084F83820022384F8393021684B6823F09A
:1021180070034B60216848682B6803434B60216853
:102128008B6823F080038B60216888686B680343A1
:102138008B6084F83920002084F8380038BD0220EC
:1021480038BD00BF002C014010390008FEE700BF71
:1021580008B50D4B1B6813B90C4A0B4B1A600A4B98
:102168001A68C31C23F00303134409498B4206D998
:1021780000F00CFD0C2303604FF0FF3008BD02494E
:102188000B60104608BD00BF8C0000201C03002017
:10219800004C002001230360014B0B60704700BF17
:1021A800040000200FB400B583B004AB53F8042B2F
:1021B80001938021064800F027FD002803DD014631
:1021C800034800F039F803B05DF804EB04B0704739
:1021D800940000202DE9F04385B004460F4643568D
:1021E80013BB042528462146ABBE04461FE03546EE
:1021F800102E28BF1025002306E014F9011B04AA9D
:102208001A4402F8101C0133AB42F6D304AA134453
:10221800002203F8102CE9464FF0040840464946CE
:10222800ABBE8046761B00E00E46002EDFD1384656
:1022380005B0BDE8F08300BF08B5FFF7CBFF08BDC8
:1022480008B500F097F8024B024A9A6008BD00BF33
:1022580000ED00E00000000808B500F0B1F808BD86
:10226800F8B504460D4617461E462648FFF79AFF5E
:1022780021682548FFF796FF61682448FFF792FF19
:10228800A1682348FFF78EFFE1682248FFF78AFF1D
:1022980021692148FFF786FF61692048FFF782FF1F
:1022A800A1691F48FFF77EFFE1691E48FFF77AFF23
:1022B8001D48FFF777FF29461C48FFF773FF1C4CA2
:1022C800E16A1C48FFF76EFF216B1B48FFF76AFFA6
:1022D800E16B1A48FFF766FF15F0800F03D0394607
:1022E8001748FFF75FFF15F4004F03D03146154834
:1022F800FFF758FF1448FFF755FF06991348FFF7F3
:1023080051FFF8BD4039000850390008603900080D
:10231800703900088039000890390008A039000891
:10232800B0390008C0390008D0390008DC39000885
:1023380000ED00E0EC390008FC3900080C3A000810
:102348001C3A00082C3A00083C3A0008443A0008B5
:1023580083691A888A4207D10268033A012A05D894
:1023680002338361012070470020704700207047C6
:10237800FEE700000F4B1A6842F001021A60596824
:102388000D4A0A405A601A6822F0847222F4803298
:102398001A601A6822F480221A605A6822F4FE022F
:1023A8005A604FF41F029A604FF00062034B9A6024
:1023B800704700BF001002400000FFF800ED00E089
:1023C8001F4B5B6803F00C03042B06D0082B08D0C6
:1023D8003BBB1C4A1C4B1A6026E01A4A1A4B1A606F
:1023E80022E0174A53685268C3F38343023312F456
:1023F800803F05D1154A02FB03F3134A136013E02B
:102408000F4A526812F4003F05D0104A02FB03F34A
:102418000D4A136008E00B4A02FB03F30A4A1360F3
:1024280002E0084A084B1A60054B5B68C3F30313C4
:10243800074AD15C044A1368CB401360704700BF59
:102448000010024000127A000C00002000093D0034
:10245800883A0008F0B589B0234B9A6942F0100217
:102468009A619A6902F010020092009A9A6942F001
:1024780020029A619A6902F020020192019A9A69EF
:1024880042F004029A619A6902F004020292029AE6
:102498009A6942F008029A619B6903F00803039362
:1024A800039B124F00224FF460413846FEF7BCFAF6
:1024B8000F4C002260212046FEF7B6FA4FF4604325
:1024C8000493012605960225079504A93846FEF7C8
:1024D8002BF9602304930596079504A92046FEF777
:1024E80023F909B0F0BD00BF001002400010014000
:1024F800000C014008B500F073FAFEE700B58FB094
:102508001D481E4B0360002343608360C360036162
:10251800FFF768FB08B1FFF7EDFF0EA94FF48053F2
:1025280041F8103D1448FFF717F908B1FFF7E2FF2B
:102538001148FFF7A5FB08B1FFF7DCFF002308935C
:10254800099308A90C48FFF7A1FD08B1FFF7D2FFCE
:1025580060230193002202920392059201A9064882
:10256800FFF734FC08B1FFF7C5FF034800F04EF948
:102578000FB05DF804FB00BF6001002000040040BC
:1025880008B50B480B4B036010234360002383609E
:10259800C360036143618361C36103624362836211
:1025A800C362FDF727FF08B1FFF7A4FF08BD00BF0E
:1025B800200100200064004000B587B015484FF0A6
:1025C800804303600023436083604FF6FF72C2605C
:1025D8000361FFF707FB08B1FFF78CFF4FF40053C7
:1025E8000293002303930493059302A90948FFF774
:1025F800B3F808B1FFF77EFF002300930193694603
:102608000448FFF743FD08B1FFF774FF07B05DF812
:1026180004FB00BF9C01002000B591B00123069384
:102628004FF4803307930022089202220D920E93F2
:102638004FF4E0130F9306A8FEF720FA08B1FFF74E
:1026480059FF0F23019302210291002303934FF4B2
:1026580080620492059301A8FEF7E8FD08B1FFF730
:1026680049FFFEF735FF094BA3FB00308009FEF751
:1026780025F80420FEF738F8002211464FF0FF3005
:10268800FDF7DAFF11B05DF804FB00BFD34D62100F
:1026980008B500F099F9FDF77FFEFFF7BDFFFFF7DA
:1026A800D9FEFFF72BFFFFF76BFFFFF785FF00F061
:1026B800A1F900F08DF9FCE7704700BF00B583B0C1
:1026C800204B9A6942F001029A619B6903F0010369
:1026D8000193019B0320FDF791FF002211466FF043
:1026E8000B00FDF7A9FF002211466FF00A00FDF765
:1026F800A3FF002211466FF00900FDF79DFF00229D
:1027080011466FF00400FDF797FF002211466FF0A5
:102718000300FDF791FF002211466FF00100FDF75D
:102728008BFF002211464FF0FF30FDF785FF064A68
:10273800536823F0E06343F00073536003B05DF81F
:1027480004FB00BF00100240000001400268144B67
:102758009A4224D110B586B003F5D633DA6942F02F
:102768000072DA61DB6903F000730193019B4FF497
:10277800006302930023039304930A4C02A92046A2
:10278800FDF7D2FF4FF480530293022303930323F0
:10279800059302A92046FDF7C7FF06B010BD704794
:1027A800006400400008014000B587B00368B3F139
:1027B800804F14D103F50433DA6942F00102DA617B
:1027C800DB6903F001030093009B012302930023BC
:1027D8000393049302A90A48FDF7A6FF0CE0094AEF
:1027E800934209D1084BDA6942F00202DA61DB69E7
:1027F80003F002030193019B07B05DF804FB00BFDF
:1028080000080140000400400010024002680C4B20
:102818009A4214D100B585B0102300930223019386
:10282800039369460748FDF77FFF074A536823F477
:10283800406343F40063536005B05DF804FB7047E0
:1028480000040040000C014000000140704700BF38
:10285800FEE700BFFEE700BFFEE700BFFEE700BFE0
:10286800704700BF704700BF704700BF08B5FDF74D
:10287800A5FDFDF755FF08BD08B54FF40051024806
:10288800FEF7ECF808BD00BF0010014008B54FF492
:102898007A7300221146024800F002F908BD00BF11
:1028A8008128000800B583B00648FFF77BFC064B7B
:1028B8001B685B6A019301990448FFF773FC03B036
:1028C8005DF804FB983A00089C010020A83A00082B
:1028D80008B50548FEF716FF642300221146034891
:1028E80000F0DEF808BD00BF9C010020AD280008FC
:1028F80010B504460378012B09D143783BB1002277
:102908004FF480411F48FEF78FF800236370237847
:102918004BB963783BB901224FF480411948FEF75F
:1029280083F8012363702378022B06D14FF480418A
:102938001448FEF793F801236370A378012B09D19B
:10294800E3783BB100224FF400410E48FEF76CF8E3
:102958000023E370A3784BB9E3783BB901224FF425
:1029680000410848FEF760F80123E370A378022BC2
:1029780006D14FF400410348FEF770F80123E370D5
:1029880010BD00BF001001400122014B9A70704732
:10299800100000200222014B1A707047100000201E
:1029A80008B5642300220549054800F079F800229B
:1029B8004FF440410348FEF737F808BD10000020E7
:1029C800F92800080010014008B500F051F808BDCA
:1029D80008B500F085F808BD08B500F0ADF808BDE9
:1029E80008B501224FF480410148FEF71DF808BDE3
:1029F8000010014008B5FFF749FF00F021F8FFF784
:102A080067FFFFF7CDFFFFF7BFFFFFF7C3FF08BD65
:102A180042680368C82101FB0233036042F20F7267
:102A2800934202DD4FF0FF324260002B01DC0122AD
:102A38004260024A12685363704700BF6001002079
:102A480008B5322300220749074800F029F807484B
:102A5800036842F21072DA62C26000215963FFF71C
:102A6800DFFA08BD14000020192A000860010020C0
:102A780030B400230EE0094C9900CA18950060197B
:102A88000022625142600272C260284620440261FC
:102A98000133DBB20F2BEED930BC7047D8010020D0
:102AA800F0B5002417E0274604EB8406B5000B4E6A
:102AB8003544ED686DB934464FEA870E0EEB0705CD
:102AC800AE00A519A2516B6000232B72E860296142
:102AD800F0BD0134E4B20F2CE5D9F0BDD8010020D7
:102AE80070B5002422E004EB84029300114A1344D9
:102AF800DB68CBB104EB840293000E4A13441B7AC3
:102B080093B1A10021448A000A4E1644013B337256
:102B1800F36830699847736833B904EB8405AB00F0
:102B2800044A13440022DA600134E4B20F2CDAD9E3
:102B380070BD00BFD801002070B400231FE003EB74
:102B48008300820010480244D268B2B103EB8300CC
:102B580082000D48825852B904469A00D518A80038
:102B680025186E682650287A411C297205E003EB67
:102B780083018800013A04490A500133DBB20F2B64
:102B8800DDD970BC704700BFD8010020014B186820
:102B9800704700BF1C00002070B5002A9AB0054697
:102BA8002DDB14461A464FF4027300910491ADF8D8
:102BB8000C304FF6FF760FD0013C1E9B69460294FD
:102BC8000594ADF80E6000F013F9421C10DB009B71
:102BD80000221A701AB070BD1E9B694602940594B3
:102BE800ADF80E6000F004F9431C04DB1AB070BDA8
:102BF8008B232B60EBE78B232B601AB070BD8B23E4
:102C080003604FF0FF30F1E710B5064C82B0009337
:102C1800246813460A4601462046FFF7BDFF02B066
:102C280010BD00BF1C0000202DE9F84F8E680C462F
:102C38009E421F46904612D88B8913F4906F10D18C
:102C4800354620682A46414600F09AFCA368226867
:102C58009E1B1544A66025600020BDE8F88F1E461F
:102C6800EEE74D692268096905EB4505C1EB020AE3
:102C7800814605EBD5750AF101006D103844A8426C
:102C88002A4684BF05462A465B0510D511464846A4
:102C980000F020FD8346F8B15246216900F0FAFBA6
:102CA800A38923F4906343F08003A38104E048469A
:102CB80000F06EFD834658B1CAEB05030BEB0A0022
:102CC80065613E46C4F810B02060A3603D46B9E790
:102CD8002169484600F0B8FC0C23C9F80030A389E4
:102CE8004FF0FF3043F04003A381BDE8F88F00BFE9
:102CF8002DE9F04F936883B09046002B72D04FF0C7
:102D080000090D464C468346166808688B68002CF7
:102D180045D09C421F469A4646D3AB8913F4906F20
:102D28002DD06F69296907EB4707C1EB000A07EB4C
:102D3800D777601C7F105044B8423A4684BF074694
:102D48003A465B0533D51146584600F0C3FC0028C7
:102D580037D052462969019000F09CFBAA89019B53
:102D680022F4906242F08002AA81CAEB070203EBC8
:102D78000A006F61A24627462B612860AA60524666
:102D8800494600F0FDFBD8F80820AB682868DB1B33
:102D98005044141BAB602860C8F8084014B3D6F838
:102DA800009074680836B2E72746A246E7E7584617
:102DB80000F0EEFC03460028D7D12969584600F0F8
:102DC80043FC0C23CBF80030AB89002243F04003CE
:102DD8004FF0FF30AB81C8F80820C8F8042003B0D2
:102DE800BDE8F08F0020C8F8040003B0BDE8F08FFC
:102DF8002DE9F04F0F4689899DB00C069246039342
:102E0800804603D53B69002B00F0F78030238DF80E
:102E18002A309AF80030002120227F4DDFF8FC91FB
:102E280009918DF82920002B00F08C80252B544621
:102E380003D117E0252B00F08E8014F8013F002BFA
:102E4800F8D1B4EB0A0B7DD052465B463946404672
:102E5800FFF7EAFE013075D0099B22785B4409939D
:102E6800002A6FD000224FF0FF31631C04920792B2
:102E780006928DF853201A920591012405E0049AD0
:102E8800401B04FA00F010430490197805226248A8
:102E98009A4600F0B9FA0AF101030028EFD1049B21
:102EA800D80644BF20228DF8532019079AF800103D
:102EB80044BF2B228DF853202A296FD0A1F130026C
:102EC800092A0BD8079B1AF8011F03EB830302EBAF
:102ED8004303A1F13002092AF5D907932E2945D0D9
:102EE80003224E4800F090FA50B10499C9EB000053
:102EF800402202FA00F041EA00030AF1010A0493B1
:102F08009AF800300622194645488DF828300AF10B
:102F1800010A00F079FA002865D0424BFBB103ABF7
:102F280000933A46404B04A94046AFF3008006465A
:102F3800721C07D0099B334409939AF80030002B80
:102F48007FF474AFBB895B0654BF09984FF0FF301C
:102F58001DB0BDE8F08FB4EB0A0B83D074E7039B78
:102F6800073323F0070308330393E3E79AF80110C4
:102F78002A291FD0A1F130020023092A0AF1010AE7
:102F88000593ADD81AF8011F03EB830302EB430343
:102F9800A1F13002092AF5D90593A1E7039A11682E
:102FA80004320029039218DB07919AF801100AF1FC
:102FB800010A93E7039B0AF102001A680433002A06
:102FC8000393B8BF4FF0FF330592AEBF9AF80210D3
:102FD8009AF802100593824682E7494243F00203B9
:102FE80007910493E1E703AB00933A460E4B04A91B
:102FF800404600F0B5F806469AE7402100F06AFB23
:103008003860386110B140237B61FFE60C23C8F8B3
:1030180000304FF0FF309BE7B03A0008B83A00089C
:10302800BC3A000800000000312C00082DE9F047E8
:103038000D690C46896891468D422A46B8BF0A46F2
:10304800C9F8002094F8431006461F46DDF8208092
:1030580011B10132C9F80020236899065DD5D9F865
:1030680000200232C9F80020236813F0060F194621
:103078001DD1E1688A1A002AD8BF194617DD04F164
:10308800190A002505E0E368D9F800209B1AAB422D
:103098000CDD0123524639463046C047013005F160
:1030A8000105F0D14FF0FF30BDE8F087216894F8B2
:1030B8004330003318BF01238A060AD5E2183021AD
:1030C80082F8431094F845105A1C224482F84310A1
:1030D800023304F1430239463046C0470130E1D09B
:1030E800236803F00603042B29D0A36822699342BE
:1030F800C8BF4FF000092FDD9B1A99441A340025E8
:1031080001E04D4528D00123224639463046C047C4
:10311800013005F10105F4D1C4E713F0060F08D119
:10312800E168D9F800208A1A002AD8BF1946A6DC17
:10313800BDE794F84330003318BF0123C9E7D9F835
:103148000000E168A3682269091A934221EAE1793B
:10315800D2DCB9F1000FD1D10020BDE8F08700BF63
:103168002DE9F0430C46097E85B06E2906461746C0
:10317800984604F1430C0C985AD01AD8632900F0E9
:10318800128100F2D68000295CD0582940F0F580E1
:1031980084F84510226803681506DFF864E203F135
:1031A80004011ED4550653BF1B6801601B880160CB
:1031B80019E0732900F0CF807ED86F2900F0E480F1
:1031C800702940F0DA80226842F0200222607823D9
:1031D80084F8453003681506DFF828E203F1040196
:1031E800E0D51B680160D00744BF42F0200222608E
:1031F800002B40F090802268102122F020022260EB
:10320800002284F8432060680028A060C0F288800B
:10321800226822F004022260002B62D1002840F0CC
:103228008180654608296AD0C5EB0C0323610CE050
:1032380023681A0640F1D58003686269191D016088
:103248001B681A60654600232361CDF800803B4661
:1032580003AA21463046FFF7E9FE013021D02A466D
:10326800236939463046C04701301AD0236803988D
:1032780013F0020FE36819D01A1A002A16DD04F1B8
:103288001909002504E0E36803981A1AAA420DDD1B
:1032980001234A4639463046C047013005F1010549
:1032A800F1D14FF0FF3005B0BDE8F0839842B8BFC8
:1032B800184605B0BDE8F083752965D078295CD13A
:1032C800226884E761682D200029C3F10003A1600A
:1032D80084F8430021DB22F00402DFF824E12260B5
:1032E8000A216546B3FBF1F201FB12331EF8030015
:1032F800134605F8010D002AF4D1082994D1236852
:10330800D90791D5626823699A428DDC302305F884
:10331800013C013D88E7102172E7DFF8E4E00A216B
:10332800002BDED19EF8003004F1420584F84230CB
:1033380078E7642901D069291FD122680368150636
:1033480003F104013AD51B680160002BBADBDFF8F2
:10335800B0E00A2157E703686268191D01601D681B
:103368000021284600F050F8002846D0401B606035
:103378002061002384F8433067E7012384F8421072
:10338800236104F14205F4E723681A061ED5036891
:103398001A1D1B680260227EDFF864E06F2A14BFE2
:1033A8000A2108212CE703680122191D1B6804F172
:1033B8004205016084F842302261DAE7550653BFBE
:1033C8001B680160B3F900300160BEE713F0400FDD
:1033D800036803F1040215BF02601B681B880260C2
:1033E800D9E713F0400F0368626903F10401016033
:1033F8001B6814BF1A801A6024E76068B8E700BF2A
:10340800C43A0008D83A0008830770B4CDB23DD05A
:10341800531E02B30278AA421ED0421C04E0D3B164
:103428000478013BAC4217D012F0030F104602F1AA
:103438000102F4D1032B11D853B30278AA420BD05E
:103448000344421C02E00178A94205D09342104689
:1034580002F10102F7D1002070BC704704460E0249
:1034680006F47F462E4346EA064622682046724006
:10347800A2F1013121EA020212F0803F04F10404B2
:10348800DBD1043B032B2046EFD8D5E71346D1E721
:103498001846E1E7844641EA000313F0030349D1E3
:1034A800403A23D30B6803604B6843608B688360A2
:1034B800CB68C3600B6903614B6943618B698361A6
:1034C800CB69C3610B6A03624B6A43628B6A83628E
:1034D800CB6AC3620B6B03634B6B43638B6B836376
:1034E800CB6BC36340304031403ADBD230320BD330
:1034F8000B6803604B6843608B688360CB68C3606C
:1035080010301031103AF3D20C3205D351F8043B85
:1035180040F8043B043AF9D2043208D0D2071CBF61
:1035280011F8013B00F8013B01D30B88038060468A
:10353800704700BF082A13D38B07B1D010F00303DC
:10354800AED0C3F10403D21ADB071CBF11F8013B4C
:1035580000F8013BA4D331F8023B20F8023B9FE777
:10356800043AD9D3013A11F8013B00F8013BF9D2EA
:103578000B7803704B7843708B7883706046704784
:103588008842F0B50DD98B1898420AD28118002AC2
:1035980051D09A1A13F8014D934201F8014DF9D10F
:1035A800F0BD0F2A48D941EA00039B0746D11546CA
:1035B80000F1100401F1100353F8106C103D44F8A9
:1035C800106C53F80C6C0F2D44F80C6C53F8086C05
:1035D80004F1100444F8186C53F8046C03F1100358
:1035E80044F8146CE8D8A2F1100323F00F0302F09A
:1035F8000F0E1033BEF1030F1944034421D90E46B0
:1036080074461D1F56F8047B043C032C45F8047FC0
:10361800F8D8AEF1040424F003040434234421440C
:1036280002F0030262B1013B0A4411F8014B8A42DD
:1036380003F8014FF9D1F0BD0346F3E70346F2E77B
:10364800F0BD7246EEE700BF30B481B151F8043CDA
:103658000439002BB8BFC9181D4B1A682AB18A4211
:103668000AD908680C18A24225D04A60196030BCF3
:1036780070478B4203D81A465368002BF9D1146857
:1036880015198D420CD007D808680C189C4218D020
:1036980030BC4B60516070470C23036030BC7047EE
:1036A80009680C44111999421460E0D10ACB0C4402
:1036B80014605360DBE714685268204481E8050011
:1036C800D4E71C685B68204481E809005160CEE7B4
:1036D8001401002070B5CD1C25F0030508350C2D0C
:1036E80038BF0C25002D06463BDBA94239D82749AF
:1036F8000A6852B113685B1B04D436E023685B1B6D
:103708001AD522465468002CF8D149681F4C002964
:1037180036D02946304600F05FF8431C21D0C41C3F
:1037280024F00304A04205D0211A304600F054F8D2
:10373800013016D0256004E00B2B0DD923601C4402
:10374800256004F10B0020F00700231DC31A02D0E6
:103758005A42E25070BD70BD94420ED06368536007
:10376800EFE70C233360002070BD0B2B03D8144601
:1037780053680B60E5E71446E0E713461446F8E79C
:10378800304600F029F86060C3E700BF140100204C
:10379800F9B1F8B506461546B2B10C4600F02EF858
:1037A800854201D82046F8BD29463046FFF792FFEA
:1037B800074668B12A462146FFF76CFE3046214687
:1037C800FFF742FF3846F8BDFFF73EFF2846F8BD31
:1037D800F8BD1146FFF77EBF38B5074C00230546F4
:1037E80008462360FEF7B4FC431C00D038BD2368AC
:1037F800002BFBD02B6038BD1C01002051F8040CB5
:103808000028BEBF091851F8043CC0180438704796
:103818002E2E2F73797374656D2F7372632F7374E3
:103828006D3332663178782F73746D333266317840
:10383800785F68616C5F63616E2E63002E2E2F7354
:10384800797374656D2F7372632F73746D33326679
:103858003178782F73746D3332663178785F6861A8
:103868006C5F636F727465782E6300002E2E2F7361
:10387800797374656D2F7372632F73746D33326649
:103888003178782F73746D3332663178785F686178
:103898006C5F6770696F2E63000000000203040507
:1038A800060708090A0B0C0D0E0F10100102000084
:1038B8002E2E2F73797374656D2F7372632F737443
:1038C8006D3332663178782F73746D3332663178A0
:1038D800785F68616C5F7263632E63002E2E2F73AE
:1038E800797374656D2F7372632F73746D333266D9
:1038F8003178782F73746D3332663178785F686108
:103908006C5F74696D2E63002E2E2F737973746546
:103918006D2F7372632F73746D3332663178782F1D
:1039280073746D3332663178785F68616C5F74697F
:103938006D5F65782E630000537461636B20667257
:10394800616D653A0A000000205230203D20202594
:103958003038580A00000000205231203D20202530
:103968003038580A00000000205232203D2020251F
:103978003038580A00000000205233203D2020250E
:103988003038580A0000000020523132203D2025EE
:103998003038580A00000000204C52203D202025D5
:1039A8003038580A00000000205043203D202025D0
:1039B8003038580A0000000020505352203D20257E
:1039C8003038580A000000004653522F4641523AF8
:1039D8000A0000002043465352203D20202530385D
:1039E800580A00002048465352203D2020253038F0
:1039F800580A00002044465352203D2020253038E4
:103A0800580A00002041465352203D2020253038D6
:103A1800580A0000204D4D464152203D202530389F
:103A2800580A00002042464152203D2020253038C7
:103A3800580A00004D6973630A000000204C522F99
:103A48004558435F52455455524E3D20253038580D
:103A58000A0000005B486172644661756C745D0A17
:103A6800000000005B4275734661756C745D0A0066
:103A78005B55736167654661756C745D0A0000008B
:103A88000000000000000000010203040607080906
:103A9800636F756E746572457865630A000000008F
:103AA80025640A0043000000232D302B200000006D
:103AB800686C4C0065666745464700003031323314
:103AC8003435363738394142434445460000000012
:103AD800303132333435363738396162636465667C
:043AE80000000000DA
:103AEC0078563412900000200000000000A24A0416
:103AFC000100010000000000010000002000002077
:103B0C0000000000000000000000000000000000A9
:103B1C000000000000000000000000000000000099
:103B2C00AC3A00080000000000000000000000009B
:103B3C000000000000000000000000000000000079
:103B4C000000000000000000000000000000000069
:103B5C000000000000000000000000000000000059
:043B6C0032547698C1
:040000050800010DE1
:00000001FF
